:0400000054EF0BF0BE
:08000800046ED8CF05F0E0CF33
:1000100006F00001E9CF0CF0EACF07F0E1CF08F0DD
:10002000E2CF09F0D9CF0AF0DACF0BF0F3CF12F01C
:10003000F4CF13F0FACF14F0F5CF15F0F6CF16F099
:10004000F7CF17F000C00EF001C00FF002C010F0A3
:1000500003C011F0F2AA30EF00F0F2B4D8EF00F0D4
:100060009DA036EF00F09EB0E2EF00F0F2A63CEF6C
:1000700000F0F2B0A2EF00F09DAA42EF00F09EBAAD
:10008000A8EF01F09DA848EF00F09EB8C5EF01F081
:100090000EC000F00FC001F010C002F011C003F05C
:1000A0000CC0E9FF07C0EAFF078E08C0E1FF09C0E6
:1000B000E2FF0AC0D9FF0BC0DAFF12C0F3FF13C082
:1000C000F4FF14C0FAFF15C0F5FF16C0F6FF17C005
:1000D000F7FF045006C0E0FF05C0D8FF100073749E
:1000E000617475733A5B74696C6C5D0073746174F0
:1000F00075733A5B6672E56E5D002D535441525440
:10010000412D00002D4156425259542D00002DF62C
:1001100070706E612D2D0000666F727473E47474DC
:1001200000002D534B494654412D00002020202033
:10013000202020200000416E6765206CF673656EFC
:100140006F726400006A1AB8008E81500018800B2C
:1001500004E16D2BD8B46E2B1A7881AC02D081BA31
:1001600022D0455220E11BAA1ED081BC03D0010E33
:10017000456E02D0020E456EF8C002F0F7C001F0E5
:100180000232013202320132023201C067FF023212
:100190000230300B006E6650CF0B0010666EF8C058
:1001A000FAF0F7C0F9F081500000F29048EF00F04B
:1001B000D59EAB888194F29448EF00F09EA8FED7BC
:1001C000AD6E1200F70ECF6ECE6A0400202A2050CA
:1001D000090825E2206A0101796B7951030818E3C7
:1001E000036A7951380FE96E000E0320EA6EEF5270
:1001F0000DE0036A7951380FE96E000E0320EA6EB4
:10020000EF6A7951100DF3CF22F002D0792BE5D7A8
:10021000236AAB988184010E0001D0DF9D88292AD2
:100220002950140802E1296A1A8A282A28506408E9
:1002300002E1286A1A86452C3CD01CB403D01C84E9
:10024000476A1C96FA51EC5D1FE303E1EB51F95D3F
:100250001BE24650F927000EFA23FAC002F0F9C05B
:1002600001F00232013202320132023201C067FF74
:1002700002320230300B006E6650CF0B0010666EFB
:10028000F92BD8B4FA2B15D0030E456EECC002F052
:10029000EBC001F00232013202320132023201C0FF
:1002A00067FF02320230300B006E6650CF0B001039
:1002B000666E455002083DE11CB603D01C86476AB5
:1002C0001C94EE51FA5D20E303E1F951ED5D1CE26F
:1002D0004650F95F000EFA5BFAC002F0F9C001F077
:1002E0000232013202320132023201C067FF0232B1
:1002F0000230300B006E6650CF0B0010666EF95165
:10030000D8B4FA07F90715D0030E456EEEC002F017
:10031000EDC001F00232013202320132023201C07C
:1003200067FF02320230300B006E6650CF0B0010B8
:10033000666E9E9048EF00F09EAAFED7ABCF19F0F4
:10034000AECF01F019A202D0AB98AB88B4EF01F0A8
:10035000036A35502D0FE96E000E0320EA6EEACFD6
:100360007CF1E9CF7BF1E8D77CC1EAFF7BC1E9FFF3
:1003700001C0EFFF352A3550020804E12E502D5CF4
:1003800001E11A8E9E9A48EF00F02350000A07E020
:10039000010A1AE0030A21E0010A2FE049D02B529A
:1003A00002E1000E01D0010E800DF350040F010197
:1003B000796F000E1BB4010E400DF350792779516F
:1003C0000001FCDE232A35D0030E22240101796FBF
:1003D00079510001F3DE232A2CD02250222A036A0D
:1003E0000B0FE96E010E0320EA6EEFCF79F10101E8
:1003F00079510001E3DE232A1CD022500F0B0FE0BD
:100400002250222A036A0B0FE96E010E0320EA6EC6
:10041000EFCF79F1010179510001D0DE08D09D982C
:10042000020ECCDE3F0E2216356A366AD58E01D01A
:10043000226A9E9848EF00F06D6F746F723A25350E
:100440006C752072706D2E00766F6C2E543A2535C7
:100450006C75206C69742E002D2D2D2D2D2D2D2DBC
:100460002D2D2D2D2D2D2D2D0000524F4C42412094
:100470005356454E534B41204142000032336532C2
:10048000354B32324D5A312E302E63004261747436
:10049000657269202B2532752E257520762E000079
:1004A0006175743A202020666C6F636B6E696E67AD
:1004B0000000766F6C2E543A25356C75206C69748B
:1004C0002E00766F6C2E423A25356C75206C69745F
:1004D0002E002D2D666C6F636B61722025336C7559
:1004E000202D2D002D2D2D2D2D2D2D2D2D2D2D2D76
:1004F0002D2D2D2D00002D25336C7520732E2D00F4
:100500006175743A2020204D61736B6F5A6F6C6C6B
:100510000000766F6C2E543A25356C75206C69742A
:100520002E00766F6C2E423A25356C75206C6974FE
:100530002E002D2D2D66796C6C6572204D5A2D2D57
:100540002D2D00002D2D2D74F66D6D6572204D5AE8
:100550002D2D2D2D00002D2D2D2D2D2D2D2D2D2D25
:100560002D2D2D2D2D2D00002D2D4861737425323C
:1005700075002D2D2D25317520732E2D00006D61F8
:100580006E75656C6C74000072656A656B7470756D
:100590006D7000002D2D2D2D2D2D2D2533752073E3
:1005A000656B2E002D2D2D2D2D2D2D2533752073B2
:1005B000656B2E0020282D20202B29006D616E7583
:1005C000656C6C740000736B7261706F7200202038
:1005D000202020202020203C2D2030202D3E0000F7
:1005E000202020205B4F5054494F4E5D0000696E23
:1005F000202620757467E56E6761720052656A6532
:100600006B7470756D7000002D2D2D2D2D2D2D2DE1
:100610002D2D2D2D2D2D2D2D0000203C2D20202D7C
:100620003E200000202020205B4F5054494F4E5D5B
:100630000000504D2D76656E7420632D72F67200A9
:100640002D2D2D2D2D2D2D2D2D2D2D2D2D2D2D2DDA
:100650000000504D2D76656E74204D5A00002D2DF2
:100660002D2D2D2D2D2D2D2D2D2D2D2D2D2D000014
:1006700072656A656B742076656E742E00002D2D90
:100680002D2D2D2D2D2D2D2D2D2D2D2D2D2D0000F4
:1006900050756D702074696C6C20504D00002D2DCC
:1006A0002D2D2D2D2D2D2D2D2D2D2D2D2D2D0000D4
:1006B0004D5A2D696E2076656E7400002D2D2D2DFE
:1006C0002D2D2D2D2D2D2D2D2D2D2D2D0000544971
:1006D00020262061766C75667420312632002D2D1F
:1006E0002D2D2D2D2D2D2D2D2D2D2D2D2D2D000094
:1006F0006B6F6C76676976206C69207369640000A3
:100700002D2D2D2D2D2D2D2D2D2D2D2D2D2D2D2D19
:1007100000006B6F6C766769762073742073696470
:1007200000002D2D2D2D2D2D2D2D2D2D2D2D2D2D53
:100730002D2D0000736F6E617267697600002D2D9C
:100740002D2D2D2D2D2D2D2D2D2D2D2D2D2D000033
:1007500072656A656B742076616B74002D2D2D2D8A
:100760002D2D2D2D2D2D2D2D2D2D2D2D0000766196
:100770006375756D70756D7000002D2D2D2D2D2DEF
:100780002D2D2D2D2D2D2D2D2D2D000074727963E5
:100790006B002D2D2D2D2D2D2D2D2D2D2D2D2D2D78
:1007A0002D2D0000496E7374E46C6C6E696E676188
:1007B000720052656A656B7474696D6572002532EA
:1007C000753A2073656B756E6465720020282D2064
:1007D00020202B2900004B616C2E207661727674EC
:1007E000616C000076E47264653A253375007270BE
:1007F0006D3A2025346C750020282D2020202B29CF
:1008000000004B616C2E20766F6C796D6769760005
:1008100076E47264653A25336C7500007265663A59
:100820002025356C750020282D2020202B29000044
:10083000546F742E20766F6C796D00006C6974654E
:10084000723A25356C75000020282D2020202B2998
:10085000000042617474657269202B2532752E2563
:100860007520762E00006B616C2E76E47264653A1A
:1008700025336C75000020282D2020202B29000016
:1008800072616D702070726F7076656E742E0000EC
:1008900020282D2020202B2900004D5A2D6861731F
:1008A000746967686574206E6572000076E472642E
:1008B000653A25336C75000020282D2020202B2937
:1008C00000004D5A2075707020286D696E29000057
:1008D00076E47264653A25336C75000020282D207B
:1008E00020202B2900004D5A2075707020286D6142
:1008F0007829000076E47264653A25346C7500004E
:1009000020282D2020202B2900006D616E2E2070C4
:100910006164646C617200002533753A20302D32B9
:100920003535000020282D2020202B2900002020F4
:1009300020205B4F5054494F4E5D00005061726162
:100940006D657465725B2533755D000020282D2070
:1009500020202B29000050613A253375000056E411
:100960007264655B25356C755D0020282D20202084
:100970002B2900005469642026206C697465726418
:100980006174610020282D2020202B29000074692B
:10099000643A2532752225356C752273656B00002B
:1009A0006C69743A25356C7500004175742E20769B
:1009B0006F6C796D000070726F6772616D6D65723A
:1009C000696E67005374617475733A5B4F4B5D00D9
:1009D0005374617475733A5B46454C5D00002D2D70
:1009E0002D2D2D2D6573632D2D2D2D676F2D000061
:1009F00041643A25336C752073656B3A25356C7507
:100A000000006164723A2025346C752000002533A3
:100A1000753A207469647376E47264656E006C6F75
:100A20006767616465206920656570726F6D00009D
:100A3000010EEA6E540EE96EEF500EE0020E016EEA
:100A4000006A002EFED7012EFBD7620E006E002E2C
:100A5000FED700D0EF2EF2D712000101666BF2CF65
:100A600067F1F29E61C1A9FFA69CA69EA680A85030
:100A700067BFF28E656F622D17D0612BF2CF67F1E1
:100A8000F29E61C1A9FFA69CA69EA680A85067BF42
:100A9000F28E666F66C164F165C163F163C101F0F6
:100AA00064C102F008D003D0646B65C163F163C117
:100AB00001F064C102F0000112000101546B5451B5
:100AC0003F080BE3036A54510B0FE96E010E03203C
:100AD000EA6E200EEF6E542BF2D7546B545103087C
:100AE0000BE3036A5451380FE96E000E0320EA6EDF
:100AF000010EEF6E542BF2D7216A000112000101A2
:100B0000726B736B010E746FDA6AD96A776F6A0E53
:100B1000766F010EEA6E6E0EE96E77C1E2FF76C166
:100B2000E1FF74C175F1D890E550EE02F3507223E5
:100B3000F4507323752FF7D772C1DEFF73C172F1C2
:100B4000736BD8B0732B762BD8B4772B742B74516E
:100B50000508DFE100011200D8B204D0010EEA6EF0
:100B6000740EE96E006A016A026A036A0101746B1D
:100B7000756B766B776B73517211711170112CE07C
:100B8000200E786FD8906C376D376E376F377437AB
:100B90007537763777377351775D08E17251765D37
:100BA00005E17151755D02E17051745D0FE37051A3
:100BB000745F7151D8A0713D755F7251D8A0723DBC
:100BC000765F7351D8A0733D775FD88000360136C9
:100BD00002360336782FD6D774C1EFFF75C1ECFF0C
:100BE00076C1ECFF77C1ECFF0001120001016AC081
:100BF0006BF169C06AF16D6B6C6B716B706B030E9E
:100C00006F6FE80E6E6F00017ADF03C057F102C00C
:100C100056F101C055F100C054F10F0E0101616F92
:100C2000010E626F000119DF01015F6B5E6B02C094
:100C30005DF101C05CF12A6A2A50255CD8A07ED003
:100C4000D8902A34800F606F616F010E626F0001CF
:100C500004DF01015B6B5A6B02C059F101C058F10E
:100C6000D8902A34036A710FE96E000E0320EA6EF1
:100C7000EACF63F1E9CF62F1D89257C16FF156C163
:100C80006EF155C16DF154C16CF15FC173F15EC17C
:100C900072F15DC171F15CC170F100015DDF63C192
:100CA000EAFF62C1E9FF03C067F102C066F101C05B
:100CB00065F100C064F1EACF69F1E9CF68F103C0E2
:100CC0006DF102C06CF101C06BF100C06AF15BC153
:100CD00071F15AC170F159C16FF158C16EF10FDF56
:100CE00069C1EAFF68C1E9FF03C067F102C066F1AC
:100CF00001C065F100C064F1EACF6BF1E9CF6AF1A0
:100D0000D89203C06FF102C06EF101C06DF100C056
:100D10006CF10101736B726B030E716FE80E706FF3
:100D200000011ADF6BC1EAFF6AC1E9FF01C0ECFFF5
:100D3000ED5200C0EFFF2A2A01017ED7000169EFC2
:100D40000CF001015A515C03F3CF01F0F4CF00F035
:100D50005D03F35000265B515C03F3500020026EEC
:100D600000011200016A026A006A036A01015F5110
:100D700002E15E5118E0100E606FD8905C375D376D
:100D8000003603365F51035C02E15E51005C07E30D
:100D90005E51005ED8A003065F51035ED880013625
:100DA0000236602FEAD70001120054C1C2FF120EB2
:100DB000006E002EFED7C282C2B2FED7050E006EB4
:100DC000002EFED700D001015B6BC4CF5AF1010E9B
:100DD0005D6F5C6B0001B5DFC35001010124586FEA
:100DE000000E0220596F5451030A000109E0040A61
:100DF00020E00C0A1FE0040A1EE01C0A1DE01CD0C3
:100E0000DA510101595D0FE305E10001D9510101FA
:100E1000585D09E30001D9510101585F0001DA5121
:100E20000101595B04D0000E016E026E59D0000121
:100E300003D002D001D000D0010157534DE05651EC
:100E4000595D22E303E15851555D1EE25551585D4D
:100E50005A6F565159595B6F5D6F5AC15CF15F6BA8
:100E600057C15EF100017EDF02C05BF101C05AF1A3
:100E7000010E01010124016E000E0220036E0150DB
:100E800055270350562322D05951565D1FE303E1E5
:100E90005551585D1BE25851555D5A6F595156597D
:100EA0005B6F5D6F5AC15CF15F6B57C15EF1000112
:100EB00059DF01C05AF1010E01010124016E000E3B
:100EC0000220036E0150555F0350565B55C101F07F
:100ED0005651026E05D004D058C101F059C102F03C
:100EE0000001120001015751100DF3505825216ED9
:100EF0003F0E21160001120001015F5324E0036A36
:100F000021500B0FE96E010E0320EA6E5F51EF5C7A
:100F100016E0036A21500B0FE96E010E0320EA6E02
:100F20005FC1EFFF2138006E0F0E00160050036AFC
:100F3000380FE96E000E0320EA6E010EEF6E2150AD
:100F40003E0801E3212A000112000900F6CF57F103
:100F5000F7CF58F1F5CF5FF1CFDF57C1F6FF58C19A
:100F6000F7FF0101562F01D002D00001EED700019A
:100F70001200EACF5EF1E9CF5DF101015739F009C6
:100F8000596F5927E20F5A6F320F5C6F57510F0B91
:100F90005A275A275C27E90F5B6F5B275B27563977
:100FA0000F0B5B275C275B375C375C1F5C37565148
:100FB0000F0B5C275937070E586F0A0E5B075C272B
:100FC000FDE35A075B27FDE359075A27FDE358075E
:100FD0005927FDE3010EEA6E580EE96E070E5D1506
:100FE0005D9DE926000EEA22E9505C0803E1EA2C47
:100FF00001D05D8DEF50006E08E15DBD06D05DB99A
:1010000015D05DB702D0200E03D05D875D99300EFC
:101010000026EACF57F1E9CF56F100C05FF1000199
:101020006BDF57C1EAFF56C1E9FF0101EE505DAD2C
:10103000DBD7000112000900F5520CE0F6CF57F1A2
:10104000F7CF58F1F5CF5FF157DF57C1F6FF58C121
:10105000F7FFF1D71200036A21500B0FE96E010E62
:101060000320EA6EEF50200816E0036A21500B0FB0
:10107000E96E010E0320EA6E200EEF6E2138006E3D
:101080000F0E00160050036A380FE96E000E0320A1
:10109000EA6E010EEF6E212A21500F0BDCE11200E7
:1010A00001015951016A585D03E258C100F00CD0AA
:1010B000006A080E5A6F583700365951005CD8B094
:1010C000006E01365A2FF7D700011200015056C1A9
:1010D00058F1640E0101596F0001E2DF00C056F1C2
:1010E0000150300E08E1010157A30FD057B70DD0C2
:1010F00057B9200E04D001015797579957810126FF
:1011000001C05FF10001F8DE010156C158F10A0E7D
:10111000596F0001C5DF00C056F10150300E08E1E3
:10112000010157B70AD057A108D057B9200E0001C6
:10113000012601C05FF1E0DE0101300E562756C1E5
:101140005FF10001D9DE1200006A016A0101575106
:10115000D89058B100260032013258B30026003230
:10116000013258B500260032013258B7002600324D
:10117000013258B900260032013258BB0026003235
:10118000013258BD00260032013258BF002600321D
:10119000013200012DEF0AF0030E0101576F586B69
:1011A0000001A0DE0101576B55510F0B586F5753CB
:1011B0000AE1582D08D0FA0EF66E000EF76E000107
:1011C0003ADF54D00101576B55510F0B586F5753ED
:1011D0000BE15851020808E1040EF66E010EF76E9D
:1011E000000129DF43D00101576B55510F0B586F98
:1011F00057530BE15851050808E10E0EF66E010E2B
:10120000F76E000118DF32D00101576B55510F0BFB
:10121000586F57530BE15851030808E1180EF66E4A
:10122000010EF76E000107DF21D00101576B555108
:101230000F0B586F57530BE15851040808E1220E69
:10124000F66E010EF76E0001F6DE10D00101576B4D
:1012500055510F0B586F57530AE15851060807E1D3
:101260002C0EF66E010EF76E0001E5DE0101576BE4
:101270005551F00B586F575314E15851100811E1B4
:101280002D50070B576F030E5B6FE80E5A6F5D6BA7
:1012900057C15CF1000155DD02C0DCF001C0DBF09C
:1012A00001011BA008D03C5205E11B900001DE6B40
:1012B000DD6B01010BD13C52D8B404D1565304E18B
:1012C0001B80010E3D6E33D00001DEC058F1DD51B0
:1012D000DD2BD8B4DE2B0101576F575305E158536E
:1012E00003E1010E3D6E23D00001DE5303E1DD5129
:1012F00028080BE2010156510208D8B402D00001BF
:1013000004D0140E3D6E13D00001DE5303E1DD5115
:10131000140803E2050E3D6E09D0DE5303E1DD51F2
:10132000070803E2010E3D6E01D03D6A0101576BD3
:1013300055510F0B586F575311E1582D0FD03C2CBE
:101340000DD00001DB2BD8B4DC2B1B801B86B40E28
:101350002B6E000E016EBDD0B3D00101576B5551FD
:101360000F0B586F57531BE15851020818E13C2CE2
:1013700016D00001DB51D20807E1DC51070804E177
:10138000DB51D8B4DC07DB07DB51D8B4DC07DB0763
:101390001B801B96000E016E9CD092D00101576BF2
:1013A00055510F0B586F57530FE1585105080CE179
:1013B0003C2C0AD00001DB2BD8B4DC2B1B80000EA8
:1013C000016E87D07DD00101576B55510F0B586FBF
:1013D00057530FE1585103080CE13C2C0AD000018F
:1013E000DB2BD8B4DC2B1B80000E016E72D068D0D2
:1013F0000101576B55510F0B586F57530CE1585162
:10140000040809E13C2C07D01C88000E016E000185
:1014100060D056D001015451F00B576F586B5751A3
:1014200010080BE1585309E13C50040806E13DC0A7
:1014300001F000014ED044D0010154510F0B576F01
:10144000586B572D0ED058530CE13C50020809E15F
:101450003DC057F15869000177D601503AD030D0DD
:1014600001015451F00B576F586B575140080EE172
:1014700058530CE13C50040809E10001DB2BD8B4BF
:10148000DC2B000E016E25D01BD0010154510F0B37
:10149000576F586B575104080FE158530DE13C50FA
:1014A00002080AE10001DB51D8B4DC07DB07000EBB
:1014B000016E0FD005D00101000E016E000109D0B0
:1014C00004D001010001DE6BDD6B0101000E016E35
:1014D00000011200010155515719800B596F55AF8A
:1014E00005D0541F551F542BD8B4552B57AF05D0DA
:1014F000561F571F562BD8B4572B54515603F3CFB2
:1015000001F0F4CF00F05703F35000265551560375
:10151000F3500020026E59AF05D0011E021E012AB1
:10152000D8B4022A0001E0EF10F001015A6B56C155
:1015300059F1F250006EF29E55C1A9FF59C1A8FFA2
:10154000A69CA69EA6840F01550EA76EAA0EA76E96
:10155000A682A6B2FED7A6940050F2120101582D21
:1015600019D057C15AF1552BF250006EF29E55C159
:10157000A9FF5AC1A8FFA69CA69EA6840F01550EDE
:10158000A76EAA0EA76EA682A6B2FED7A69400509A
:10159000F21201011B820001120001015591545108
:1015A000010A00011BE0030A1FE0010A23E0070A09
:1015B00027E0010A2BE0030A2FE0010A33E00F0ABB
:1015C00037E0010A3BE0030A3FE0010A43E0070A73
:1015D00047E0010A4BE0030A4FE054D01BA403D0BC
:1015E0000101558100014ED082A403D00101558133
:1015F000000148D081A603D001015581000142D0ED
:1016000082A003D00101558100013CD082AA03D001
:1016100001015581000136D082A803D00101558116
:10162000000130D082A603D00101558100012AD0EB
:1016300080A803D001015581000124D081BC03D0D2
:101640000101558100011ED081BA03D001015581ED
:10165000000118D081B803D001015581000112D0DA
:1016600081B203D00101558100010CD081B003D0BB
:1016700001015581000106D01DA003D00101558153
:10168000000100D0010155A108D0DE0EF66E000E5B
:10169000F76E0001D0DC07D00101EC0EF66E000EF3
:1016A000F76E0001C8DC1200F86AD09E078EFE0EAD
:1016B000006E060E016E020EE96E000EEA6EEE6A14
:1016C0000400002EFCD7012EFAD7196AB896050E31
:1016D000AF6EA20EAC6E900EAB6E0101536B526BEF
:1016E0000F01386B396B3A6B776A786A796A2F0E1B
:1016F000926EF30E936E800E946E810EC06E0A0E83
:10170000C16E896A8A6A8B6A280E0101546F0001D2
:1017100018EC05F0609060926094B40E2B6ED1804E
:10172000090E446E3B0E0101616F010E626F0001F4
:101730002DEC05F002C006F101C005F13D0E0101DE
:10174000616F010E626F00012DEC05F002C008F11F
:1017500001C007F1370E0101616F010E626F0001D8
:101760002DEC05F002C004F101C003F1400E0101AF
:10177000616F010E626F00012DEC05F002C002F1F5
:1017800001C001F1420E0101616F626B00012DEC9D
:1017900005F001C046F01E0E0101616F626B000191
:1017A0002DEC05F001C04DF00C0E0101616F010E32
:1017B000626F00012DEC05F002C06AF001C069F013
:1017C0006AC062F069C061F00E0E0101616F626B68
:1017D00000012DEC05F001C025F0600E0101616FE4
:1017E000010E626F00012DEC05F002C0DAF001C0BD
:1017F000D9F00101616B626B00012DEC05F001C0B5
:1018000049F04950040802E3050E496E480E0101F3
:10181000616F626B00012DEC05F001C02CF05F0ED2
:101820000101616F626B00012DEC05F002C0D8F080
:1018300001C0D7F0320E0101616F010E626F00012D
:101840002DEC05F002C0FEF001C0FDF0340E0101E8
:10185000616F626B00012DEC05F001C041F0430E99
:101860000101616F010E626F00012DEC05F002C0F5
:101870000AF101C009F1350E0101616F626B0001CF
:101880002DEC05F00150021002E01D8201D01D92E6
:10189000370ECD6ECC6AC20ED56E8B920C0E666E74
:1018A000656A646A010E636EE70E0F014917000E48
:1018B00049130409BA6EFF0EBB6E9D80F28A9D8AA1
:1018C000F2866212C00EF21200015DEC05F0F6EF36
:1018D00005F0280E0101546F000118EC05F00B0E05
:1018E0000101546F5AC056F159C055F1576B0001B0
:1018F000D5EC06F002C05AF001C059F0D8905A3029
:101900000101556F5930546F095154250001F76F8B
:1019100001010A5155210001F86FF8C002F0F7C02B
:1019200001F00232013202320132023201C067FF9D
:1019300002320230300B006E6650CF0B0010666E24
:10194000C150F00BC16E2F0E0F01386F000E396FB2
:101950003A6F030E0101546F56C056F155C055F150
:10196000576B0001D5EC06F002C056F001C055F0EF
:10197000070E0101546F58C056F157C055F1576B0F
:101980000001D5EC06F002C058F001C057F00F0E70
:101990000101546F5CC056F15BC055F1576B0001FB
:1019A000D5EC06F002C05CF001C05BF0130E010143
:1019B000546F5EC056F15DC055F1576B0001D5EC18
:1019C00006F002C05EF001C05DF0F8C0FAF0F7C0AA
:1019D000F9F001015AC055F159C054F107C100F0A6
:1019E00008C101F05B6B5A6B01C059F100C058F19E
:1019F0006D6B6C6B5AC06BF159C06AF1716B706B97
:101A000001C06FF100C06EF100017FEC05F003C072
:101A100057F102C056F101C055F100C054F1D892FF
:101A200003C06FF102C06EF101C06DF100C06CF136
:101A30000101736B726B030E716FE80E706F000122
:101A4000ACEC05F001C0F2F000C0F1F001015AC0A9
:101A500055F159C054F105C100F006C101F05B6BAE
:101A60005A6B01C059F100C058F16D6B6C6B5AC0D4
:101A70006BF159C06AF1716B706B01C06FF100C0FE
:101A80006EF100017FEC05F003C057F102C056F182
:101A900001C055F100C054F1D89203C06FF102C0EB
:101AA0006EF101C06DF100C06CF10101736B726BDE
:101AB000030E716FE80E706F0001ACEC05F001C011
:101AC000F0F000C0EFF0EF51F15D0101546F000143
:101AD000F051F2590101556F576B010E4424016E0C
:101AE000000E5721036E01C056F1576F55C15BF1CF
:101AF00054C15AF15D6F01C05CF10001A1EC06F028
:101B000002C055F101C054F102C05DF101C05CF1A9
:101B100001015F6B0A0E5E6F0001B2EC06F001502E
:101B2000EF25EB6F0250F021EC6F01015AC055F127
:101B300059C054F103C100F004C101F05B6B5A6B52
:101B400001C059F100C058F16D6B6C6B5AC06BF15C
:101B500059C06AF1716B706B01C06FF100C06EF11A
:101B600000017FEC05F003C057F102C056F101C03F
:101B700055F100C054F1D89203C06FF102C06EF16C
:101B800001C06DF100C06CF10101736B726B030E4B
:101B9000716FE80E706F0001ACEC05F001C0EEF063
:101BA00000C0EDF01F6A1AAE51EF21F01A9E1BB66D
:101BB00002D01B981B9A2D50380B006E00303C6EE3
:101BC0003C323C321F0E3C16DBC000F0DC51036E91
:101BD00003E10052D8B453D1035004E1010E005C7C
:101BE000D8B4F5D1030E035C04E1E80E005CD8B470
:101BF000F0D1030E035C04E1E90E005CD8B4E9D136
:101C0000070E035C04E1D00E005CD8B401D3070ECC
:101C1000035C04E1D10E005CD8B4FCD2070E035C77
:101C200004E1D20E005CD8B4F5D20B0E035C05E1E2
:101C3000B80E005CD8B4BDEF12F00B0E035C05E1EA
:101C4000B90E005CD8B4BDEF12F00F0E035C05E1D5
:101C5000A00E005CD8B487EF13F0130E035C05E10F
:101C6000880E005CD8B40EEF14F0170E035C05E18B
:101C7000700E005CD8B441EF14F0170E035C05E160
:101C8000710E005CD8B490EF14F0170E035C05E100
:101C9000720E005CD8B4CFEF14F0170E035C05E1B0
:101CA000730E005CD8B4CFEF14F0170E035C05E19F
:101CB000740E005CD8B4FAEF14F0170E035C05E163
:101CC000750E005CD8B433EF15F0170E035C05E118
:101CD000760E005CD8B46CEF15F0170E035C05E1CE
:101CE000770E005CD8B4A5EF15F0170E035C05E184
:101CF000780E005CD8B4DEEF15F0170E035C05E13A
:101D0000790E005CD8B417EF16F0170E035C05E1EE
:101D10007A0E005CD8B454EF16F0170E035C05E1A0
:101D20007B0E005CD8B489EF16F0170E035C05E15A
:101D30007C0E005CD8B4BEEF16F0170E035C05E114
:101D40007D0E005CD8B4F3EF16F0170E035C05E1CE
:101D50007E0E005CD8B428EF17F0170E035C05E187
:101D60007F0E005CD8B45DEF17F0170E035C05E141
:101D7000800E005CD8B4B3EF17F01B0E035C05E1D6
:101D8000580E005CD8B4B9EF17F01B0E035C05E1E8
:101D9000590E005CD8B415EF18F01B0E035C05E17A
:101DA0005A0E005CD8B499EF18F01B0E035C05E1E5
:101DB0005B0E005CD8B42CEF19F01B0E035C05E140
:101DC0005C0E005CD8B4CBEF19F01B0E035C05E190
:101DD0005D0E005CD8B454EF1AF01B0E035C05E1F5
:101DE0005E0E005CD8B416EF1BF01B0E035C05E121
:101DF0005F0E005CD8B499EF1BF01B0E035C05E18D
:101E0000600E005CD8B477EF1CF01B0E035C05E19C
:101E1000610E005CD8B458EF1DF01B0E035C05E1A9
:101E2000620E005CD8B438EF1EF01B0E035C05E1B7
:101E3000630E005CD8B4B8EF1EF01B0E035C05E126
:101E4000640E005CD8B4E3EF1EF01B0E035C05E1EA
:101E5000650E005CD8B445EF1FF01B0E035C05E176
:101E6000660E005CD8B406EF20F01B0E035C05E1A3
:101E7000670E005CD8B4D6EF20F04FEF21F00101DF
:101E8000576B586B000172EC07F0380EF66E040EBB
:101E9000F76E060E0101566F0001A5EC07F0000E6B
:101EA000E96E70C057F16FC056F1B9EC07F0420E01
:101EB000F66E040EF76E050E0101566F0001A5ECDB
:101EC00007F0010E0101576F586B000172EC07F02B
:101ED000480EF66E040EF76E060E0101566F0001F5
:101EE000A5EC07F0000EE96EE0C057F1DFC056F137
:101EF000B9EC07F0520EF66E040EF76E050E0101F6
:101F0000566F0001A5EC07F0020E0101576F586BE8
:101F1000000172EC07F0580EF66E040EF76E1BEC23
:101F200008F0030E0101576F586B000172EC07F0C7
:101F30004C50010807E36A0EF66E040EF76E1BECB8
:101F400008F036D04C50020809E37C0EF66E040E01
:101F5000F76E1BEC08F02BEC08F02AD08C0EF66E16
:101F6000040EF76E090E0101566F0001A5EC07F093
:101F70004AC056F1110E0101576F000166EC08F0DE
:101F80002E0E01015F6F00017CEC07F04BC056F193
:101F90001B0E0101576F000166EC08F09B0EF66EF8
:101FA000040EF76E030E0101566F0001A5EC07F059
:101FB000100E0101556F546B566B0001CCEC08F00C
:101FC0003E6ADB51DC1101E03E6A51EF21F051EF36
:101FD00021F00101576B586B000172EC07F0DB51E7
:101FE000E8080AE1DC51030807E1A00EF66E040ED2
:101FF000F76E1BEC08F01CD0B20EF66E040EF76EF6
:10200000060E0101566F0001A5EC07F0000EE96E07
:10201000E0C057F1DFC056F1B9EC07F0BC0EF66E28
:10202000040EF76E050E0101566F0001A5EC07F0D6
:10203000010E0101576F586B000172EC07F0C20EE0
:10204000F66E040EF76E060E0101566F0001A5EC48
:1020500007F0000EE96E66C057F165C056F1B9ECA5
:1020600007F0CC0EF66E040EF76E050E0101566FEA
:102070000001A5EC07F0020E0101576F586B00013B
:1020800072EC07F081A61DD0D20EF66E040EF76E2C
:102090000A0E0101566F0001A5EC07F0020EE96E71
:1020A000FCC057F1FBC056F1B9EC07F0E00EF66E3C
:1020B000040EF76E030E0101566F0001A5EC07F048
:1020C00006D0E40EF66E040EF76E1BEC08F03E52DE
:1020D0001DE1320E0101616F010E626F00012DECF6
:1020E00005F002C055F101C054F102C05DF101C01C
:1020F0005CF101015F6B050E5E6F0001B2EC06F052
:1021000001C051F002C052F0010E3E6E1BB60CD061
:10211000110E0101556F546F010E566F0001CCEC8A
:1021200008F001C050F00DD0020E0101556F110EE4
:10213000546F010E566F0001CCEC08F001C050F056
:102140001B8850AE01D01C8A2D0E01015F6F00016B
:102150007CEC07F0020EE96EFEC057F1FDC056F1AF
:10216000B9EC07F0FB0EF66E040EF76E040E0101DB
:10217000566F0001A5EC07F0505209E0020E3E6ECA
:10218000036A5050E8BE030651260350522252AE55
:1021900002D0526A516A52BE08D0525203E15150E5
:1021A000640803E2526A640E516E52C055F151C088
:1021B00054F10101576B050E566F00016AEF0AF0EA
:1021C00001C0FDF002C0FEF0FD51FE1105E1E66B1D
:1021D000E56BEA6BE96B1B8CF351DB5D03E1F451BA
:1021E000DC5D14E0DCC0F4F0DBC0F3F03E5002082C
:1021F0000CE1320E0101556FFEC057F1FDC056F1E2
:10220000010E586F000195EC0AF03E6A51EF21F083
:102210008284808881B005D01DB003D080988284EC
:102220000FD01DA00BD082A609D0DB51D20806E149
:10223000DC51070803E18294808802D08284808880
:102240000101576B586B000172EC07F0DB51D008AD
:102250000AE1DC51070807E1000EF66E050EF76E85
:102260001BEC08F01CD0120EF66E050EF76E060E73
:102270000101566F0001A5EC07F0000EE96EE0C009
:1022800057F1DFC056F1B9EC07F01C0EF66E050EE3
:10229000F76E050E0101566F0001A5EC07F0010E67
:1022A0000101576F586B000172EC07F0220EF66EB9
:1022B000050EF76E060E0101566F0001A5EC07F042
:1022C000000EE96E64C057F163C056F1B9EC07F037
:1022D0002C0EF66E050EF76E050E0101566F00010D
:1022E000A5EC07F0020E0101576F586B000172EC6C
:1022F00007F082A607D0320EF66E050EF76E1BECC5
:1023000008F00FD01BA407D0440EF66E050EF76E32
:102310001BEC08F006D0560EF66E050EF76E1BECA1
:1023200008F03E520FE1DB51D10807E1DC5107080C
:1023300004E144C051F0526A03D040C051F0526AE7
:10234000010E3E6E1BB60FD051C040F0110E0101C0
:10235000556F546B566B0001CCEC08F001C050F087
:102360002BEC08F082D0DB51D1084CE1DC5107089E
:1023700049E1050E0101556F110E546F566B0001B6
:10238000CCEC08F001C050F051C044F0010E4424E0
:102390000101546F680EF66E050EF76E060E566F4D
:1023A0000001A5EC07F054C156F1110E0101576F61
:1023B000000166EC08F01BBA1AD0F8C002F0F7C0B2
:1023C00001F00232013202320132023201C067FFF3
:1023D00002320230300B006E6650CF0B0010666E7A
:1023E000F8C0FAF0F7C0F9F0020E456E48681B8A93
:1023F0001CA207D01B0EDC6F5E0EDB6F3E6A51EF36
:1024000021F033D0DB51D20830E1DC5107082DE157
:1024100051C040F0020E0101556F110E546F566B02
:102420000001CCEC08F001C050F050AE02D0050E17
:102430004F6E720EF66E050EF76E030E0101566FAB
:102440000001A5EC07F040C056F1180E0101576FCE
:10245000000166EC08F0780EF66E050EF76E040EBD
:102460000101566F0001A5EC07F0505264E0020E26
:102470003E6E036A5050E8BE0306512603505222B6
:1024800052AE02D0526A516A52BE08D0525203E193
:102490005150090803E2526A090E516E1CA44BD038
:1024A000DB51D10848E1DC51070845E1EF51F15D0E
:1024B0000101546F0001F051F2590101556F576B42
:1024C000010E4424016E000E5721036E01C056F127
:1024D000576F55C15BF154C15AF15D6F01C05CF19A
:1024E0000001A1EC06F002C055F101C054F102C098
:1024F0005DF101C05CF101015F6B0A0E5E6F0001CE
:10250000B2EC06F00150EF25EB6F0250F021EC6FBA
:10251000ECC002F0EBC001F00232013202320132B3
:10252000023201C067FF02320230300B006E66508B
:10253000CF0B0010666EF351DB5D03E1F451DC5DFF
:102540001AE0DCC0F4F0DBC0F3F0526A516A3E6A74
:10255000DB51D00803E1DC5107080DE0DB51D10865
:1025600003E1DC51070807E0DB51D20803E1DC514D
:10257000070801E0809851EF21F00101576B586B7B
:10258000000172EC07F07E0EF66E050EF76E1BEC86
:1025900008F02BEC08F0010E0101576F586B000199
:1025A00072EC07F0880EF66E050EF76E1BEC08F065
:1025B0002BEC08F0020E0101576F586B000172EC12
:1025C00007F042521DE0940EF66E050EF76E070EF0
:1025D0000101566F0001A5EC07F042C056F1130E41
:1025E0000101576F000166EC08F09E0EF66E050EB5
:1025F000F76E050E0101566F0001A5EC07F01CD027
:10260000A40EF66E050EF76E070E0101566F00015F
:10261000A5EC07F041C056F1130E0101576F000100
:1026200066EC08F0AE0EF66E050EF76E050E0101B3
:10263000566F0001A5EC07F02BEC08F01BB636D066
:102640003E5205E141C051F0526A010E3E6E110E3C
:102650000101556F546F010E566F0001CCEC08F06C
:1026600001C050F0426A1C90B40EF66E050EF76E73
:102670001BEC08F0505209E0020E3E6E036A505007
:10268000E8BE030651260350522252AE02D0526ACF
:10269000516A52BE08D0525203E15150630803E21E
:1026A000526A630E516E51C041F017D0020E010103
:1026B000556F546B566B0001CCEC08F0425204E1AC
:1026C0001BB402D01C8009D0425207E11CB005D0D7
:1026D0000B0EDC6FB80EDB6F1B962BEC08F0DB519A
:1026E000B80803E1DC510B0810E03E5002080AE193
:1026F000340E0101556F576B51C056F1586B0001F4
:1027000095EC0AF03E6A526A516A51EF21F00101DC
:10271000576B586B000172EC07F0BC0EF66E050E9D
:10272000F76E1BEC08F02BEC08F0010E0101576F5F
:10273000586B000172EC07F0C60EF66E050EF76ED0
:102740001BEC08F02BEC08F0020E0101576F586BE0
:10275000000172EC07F0CE0EF66E050EF76E1BEC64
:1027600008F0100E0101556F546B566B0001CCEC54
:1027700008F001C050F03C5002081AE14D50F15DE4
:102780000101546F000E0001F2590101556F5533DC
:10279000543355335433553354C167FF5533553192
:1027A000300B006E6650CF0B0010666E32D0000109
:1027B0003C5004081AE14D50ED250101546F000E04
:1027C0000001EE210101556F553354335533543315
:1027D000553354C167FF55335531300B006E665089
:1027E000CF0B0010666E15D00001F8C002F0F7C0E4
:1027F00001F00232013202320132023201C067FFBF
:1028000002320230300B006E6650CF0B0010666E45
:10281000010100012BEC08F051EF21F00101576B91
:10282000586B000172EC07F02BEC08F0010E01016F
:10283000576F586B000172EC07F0E00EF66E050E54
:10284000F76E1BEC08F02BEC08F0020E0101576F3D
:10285000586B000172EC07F02BEC08F0030E01013D
:10286000576F586B000172EC07F02BEC08F0100E5C
:102870000101556F546B566B0001CCEC08F051EF21
:1028800021F01F6A0101576B586B000172EC07F0D1
:10289000EE0EF66E050EF76E1BEC08F02BEC08F052
:1028A000010E0101576F586B000172EC07F02BEC21
:1028B00008F0020E0101576F586B000172EC07F02F
:1028C0002BEC08F0100E0101556F110E546F566B72
:1028D0000001CCEC08F001C050F050BE0AD05050BE
:1028E000000807E2036A5050E8BE03065126035071
:1028F000522250AE11D0515002080BE1525209E160
:10290000050E1F6E170EDC6F710EDB6F526A516A77
:1029100002D0526A516A3E6A2BEC08F051EF21F066
:102920000101576B586B000172EC07F0FC0EF66E5C
:10293000050EF76E1BEC08F02BEC08F0010E010100
:10294000576F586B000172EC07F0010E0101546FD4
:102950000001CDEC0AF02BEC08F0020E0101576FDC
:10296000586B000172EC07F0080EF66E060EF76E5B
:102970001BEC08F0040E0101556F440E546F566BAA
:102980000001CCEC08F01CA802D01C981B741A0E95
:10299000F66E060EF76E1BEC08F051EF21F0010108
:1029A000576B586B000172EC07F02BEC08F0010E2E
:1029B0000101576F586B000172EC07F0240EF66EA0
:1029C000060EF76E1BEC08F02BEC08F0020E01016E
:1029D000576F586B000172EC07F02BEC08F0060EF5
:1029E0000101556F440E546F566B0001CCEC08F09A
:1029F00051EF21F00101576B586B000172EC07F0A9
:102A0000320EF66E060EF76E1BEC08F02BEC08F09B
:102A1000010E0101576F586B000172EC07F0030EB5
:102A20000101546F0001CDEC0AF02BEC08F0020E0E
:102A30000101576F586B000172EC07F0400EF66E03
:102A4000060EF76E1BEC08F0040E0101556F440EE4
:102A5000546F566B0001CCEC08F01CA802D01C98F7
:102A6000817651EF21F00101576B586B000172EC38
:102A700007F0520EF66E060EF76E1BEC08F02BEC0C
:102A800008F0010E0101576F586B000172EC07F05E
:102A9000040E0101546F0001CDEC0AF02BEC08F09C
:102AA000020E0101576F586B000172EC07F05E0EC9
:102AB000F66E060EF76E1BEC08F0040E0101556F62
:102AC000440E546F566B0001CCEC08F01CA802D0E9
:102AD0001C98827051EF21F00101576B586B000177
:102AE00072EC07F0700EF66E060EF76E1BEC08F037
:102AF0002BEC08F0010E0101576F586B000172ECCE
:102B000007F0050E0101546F0001CDEC0AF02BEC2B
:102B100008F0020E0101576F586B000172EC07F0CC
:102B20007E0EF66E060EF76E1BEC08F0040E010129
:102B3000556F440E546F566B0001CCEC08F01CA886
:102B400002D01C98827A51EF21F00101576B586B2B
:102B5000000172EC07F0900EF66E060EF76E1BEC9D
:102B600008F02BEC08F0010E0101576F586B0001C3
:102B700072EC07F0060E0101546F0001CDEC0AF073
:102B80002BEC08F0020E0101576F586B000172EC3C
:102B900007F09E0EF66E060EF76E1BEC08F0040EA4
:102BA0000101556F440E546F566B0001CCEC08F0D8
:102BB0001CA802D01C98827851EF21F00101576BBC
:102BC000586B000172EC07F0B00EF66E060EF76E51
:102BD0001BEC08F02BEC08F0010E0101576F586B4D
:102BE000000172EC07F0070E0101546F0001CDECFB
:102BF0000AF02BEC08F0020E0101576F586B000130
:102C000072EC07F0BC0EF66E060EF76E1BEC08F0C9
:102C1000040E0101556F440E546F566B0001CCEC4D
:102C200008F01CA802D01C98827651EF21F0010117
:102C3000576B586B000172EC07F0CE0EF66E060E65
:102C4000F76E1BEC08F02BEC08F0010E0101576F3A
:102C5000586B000172EC07F0080E0101546F00017F
:102C6000CDEC0AF02BEC08F0020E0101576F586B07
:102C7000000172EC07F0DE0EF66E060EF76E1BEC2E
:102C800008F0040E0101556F440E546F566B00019D
:102C9000CCEC08F01CA806D01C98807880A8829400
:102CA00080B8828451EF21F00101576B586B00010D
:102CB00072EC07F0F00EF66E060EF76E1BEC08F0E5
:102CC0002BEC08F0010E0101576F586B000172ECFC
:102CD00007F0090E0101546F0001CDEC0AF02BEC56
:102CE00008F0020E0101576F586B000172EC07F0FB
:102CF000000EF66E070EF76E1BEC08F0060E0101D3
:102D0000556F440E546F566B0001CCEC08F051EF38
:102D100021F00101576B586B000172EC07F0120EA5
:102D2000F66E070EF76E1BEC08F02BEC08F0010EA8
:102D30000101576F586B000172EC07F00A0E010198
:102D4000546F0001CDEC0AF02BEC08F0020E0101EB
:102D5000576F586B000172EC07F0220EF66E070EEB
:102D6000F76E1BEC08F0060E0101556F440E546F10
:102D7000566B0001CCEC08F051EF21F00101576BCC
:102D8000586B000172EC07F0340EF66E070EF76E0A
:102D90001BEC08F02BEC08F0010E0101576F586B8B
:102DA000000172EC07F00B0E0101546F0001CDEC35
:102DB0000AF02BEC08F0020E0101576F586B00016E
:102DC00072EC07F03E0EF66E070EF76E1BEC08F085
:102DD000060E0101556F440E546F566B0001CCEC8A
:102DE00008F051EF21F00101576B586B000172ECB4
:102DF00007F0500EF66E070EF76E1BEC08F02BEC8A
:102E000008F0010E0101576F586B000172EC07F0DA
:102E10000C0E0101546F0001CDEC0AF02BEC08F010
:102E2000020E0101576F586B000172EC07F05C0E47
:102E3000F66E070EF76E1BEC08F0060E0101556FDB
:102E4000440E546F566B0001CCEC08F051EF21F0AA
:102E50000101576B586B000172EC07F06E0EF66EB5
:102E6000070EF76E1BEC08F02BEC08F0010E0101C9
:102E7000576F586B000172EC07F00D0E0101546F93
:102E80000001CDEC0AF02BEC08F0020E0101576FA7
:102E9000586B000172EC07F07A0EF66E070EF76EB3
:102EA0001BEC08F0060E0101556F440E546F566B73
:102EB0000001CCEC08F051EF21F0070E0101546F36
:102EC00058C056F157C055F1576B0001D5EC06F0CC
:102ED00002C058F001C057F05850020807E2FF0A3C
:102EE00003E15750200802E21D8008D05850010825
:102EF00005E303E15750F30801E31D900101576B0F
:102F0000586B000172EC07F08C0EF66E070EF76E30
:102F10001BEC08F02BEC08F0010E0101576F586B09
:102F2000000172EC07F00E0E0101546F0001CDECB0
:102F30000AF02BEC08F0020E0101576F586B0001EC
:102F400072EC07F0920EF66E070EF76E1BEC08F0AF
:102F5000060E0101556F440E546F566B0001CCEC08
:102F600008F051EF21F0170EDC6F700EDB6F51EFA0
:102F700021F01BAA06D0070EDC6FD10EDB6F51EFDC
:102F800021F00101576B586B000172EC07F0A40EA1
:102F9000F66E070EF76E1BEC08F02BEC08F0010E36
:102FA0000101576F586B000172EC07F02BEC08F031
:102FB000020E0101576F586B000172EC07F02BEC09
:102FC00008F0100E0101556F110E546F566B000181
:102FD000CCEC08F001C050F050BE0AD050500008B0
:102FE00007E2036A5050E8BE0306512603505222FE
:102FF00050AE17D05150020808E1525206E11B0EA4
:10300000DC6F590EDB6F526A516A5150050806E1B8
:10301000525204E11C82526A516A02D0526A516AC9
:103020003E6A2BEC08F051EF21F00101576B586B11
:10303000000172EC07F0B20EF66E070EF76E1BEC95
:1030400008F02BEC08F0010E0101576F586B0001DE
:1030500072EC07F051C056F1110E0101576F0001DB
:1030600066EC08F0C10EF66E070EF76E0A0E01014F
:10307000566F0001A5EC07F02BEC08F0020E0101E1
:10308000576F586B000172EC07F02BEC08F03E52C2
:103090000DE1340E0101616F626B00012DEC05F052
:1030A00002C052F001C051F0010E3E6E030E01014C
:1030B000556F110E546F010E566F0001CCEC08F0E5
:1030C00001C050F0CC0EF66E070EF76E1BEC08F048
:1030D000505209E0020E3E6E036A5050E8BE0306ED
:1030E00051260350522252AE02D0526A516A52BE49
:1030F00008D0525203E15150630803E2526A630E52
:10310000516E51C041F0DB51590803E1DC511B08FD
:103110000EE03E5002080AE1340E0101556F576B74
:1031200051C056F1586B000195EC0AF03E6A51EF20
:1031300021F00101576B586B000172EC07F0D60EBD
:10314000F66E070EF76E1BEC08F02BEC08F0010E84
:103150000101576F586B000172EC07F0E40EF66E38
:10316000070EF76E060E0101566F0001A5EC07F081
:1031700051C056F1130E0101576F000166EC08F0C3
:103180002BEC08F0020E0101576F586B000172EC36
:1031900007F0EE0EF66E070EF76E050E0101566F84
:1031A0000001A5EC07F0010EE96E70C057F16FC089
:1031B00056F1B9EC07F02BEC08F03E520DE1480E49
:1031C0000101616F626B00012DEC05F002C052F04D
:1031D00001C051F0010E3E6E030E0101556F110E3C
:1031E000546F010E566F0001CCEC08F001C050F096
:1031F000F80EF66E070EF76E1BEC08F0505209E061
:10320000020E3E6E036A5050E8BE0306512603507C
:10321000522252AE02D0526A516A52BE05D052506A
:10322000000802E2526A516851C02CF0DB515A0882
:1032300003E1DC511B080EE03E5002080AE1480E93
:103240000101556F576B51C056F1586B000195EC59
:103250000AF03E6A51EF21F00101576B586B0001F3
:1032600072EC07F0020EF66E080EF76E1BEC08F01B
:103270002BEC08F0010E0101576F586B000172EC46
:1032800007F0100EF66E080EF76E060E0101566F6F
:103290000001A5EC07F0020EE96E52C057F151C0D3
:1032A00056F1B9EC07F02BEC08F0020E0101576F54
:1032B000586B000172EC07F01C0EF66E080EF76EEC
:1032C000050E0101566F0001A5EC07F0000EE96E36
:1032D00056C057F155C056F1B9EC07F02BEC08F089
:1032E0003E520EE1600E0101616F010E626F00013E
:1032F0002DEC05F002C052F001C051F0010E3E6EFF
:10330000030E0101556F110E546F010E566F00012F
:10331000CCEC08F001C050F0260EF66E080EF76EE9
:103320001BEC08F0505209E0020E3E6E036A50504A
:10333000E8BE030651260350522252AE02D0526A12
:10334000516A52BE0CD05250000809E2FF0A03E154
:103350005150F40804E2010E526EF40E516E52C048
:10336000DAF051C0D9F0DB515B0803E1DC511B08F6
:1033700010E03E5002080CE1600E0101556F52C092
:1033800057F151C056F1010E586F000195EC0AF04B
:103390003E6A51EF21F00101576B586B000172EC4E
:1033A00007F0300EF66E080EF76E1BEC08F02BECF3
:1033B00008F0010E0101576F586B000172EC07F025
:1033C0003C0EF66E080EF76E060E0101566F0001F8
:1033D000A5EC07F0000EE96E52C057F151C056F14E
:1033E000B9EC07F02BEC08F0020E0101576F586B97
:1033F000000172EC07F02BEC08F03E520EE10C0ECF
:103400000101616F010E626F00012DEC05F002C039
:1034100052F001C051F0010E3E6E030E0101556FD6
:10342000110E546F010E566F0001CCEC08F001C074
:1034300050F0480EF66E080EF76E1BEC08F0505276
:1034400009E0020E3E6E036A5050E8BE03065126A4
:103450000350522252AE02D0526A516A52BE0CD070
:1034600052504D0809E2FF0A03E15150200804E2DE
:103470004E0E526E200E516EDB515C0803E1DC51A2
:103480001B0810E03E5002080CE10C0E0101556FC4
:1034900052C057F151C056F1010E586F000195EC22
:1034A0000AF03E6A51EF21F00101576B586B0001A1
:1034B00072EC07F0520EF66E080EF76E090E01015F
:1034C000566F0001A5EC07F04AC056F1110E01013C
:1034D000576F000166EC08F02E0E01015F6F0001CE
:1034E0007CEC07F04BC056F11B0E0101576F000139
:1034F00066EC08F0610EF66E080EF76E030E010121
:10350000566F0001A5EC07F0010E0101576F586BD3
:10351000000172EC07F0660EF66E080EF76E0A0EEA
:103520000101566F0001A5EC07F0020EE96E52C0D2
:1035300057F151C056F1B9EC07F02BEC08F0020E30
:103540000101576F586B000172EC07F02BEC08F08B
:103550003E520EE1400E0101616F010E626F0001EB
:103560002DEC05F002C052F001C051F0010E3E6E8C
:10357000030E0101556F110E546F010E566F0001BD
:10358000CCEC08F001C050F0760EF66E080EF76E27
:103590001BEC08F050521CE0020E3E6E036A5050C5
:1035A000E8BE030651260350522252C002F051C019
:1035B00001F00232013202320132023201C067FFF1
:1035C00002320230300B006E6650CF0B0010666E78
:1035D00052AE02D0526A516A52BE0CD0525002080A
:1035E00009E2FF0A03E15150E70804E2030E526EBC
:1035F000E70E516E52C002F151C001F1DB515D087E
:1036000003E1DC511B0810E03E5002080CE1400EC3
:103610000101556F52C057F151C056F1010E586F5C
:10362000000195EC0AF03E6A51EF21F00101576B61
:10363000586B000172EC07F0800EF66E080EF76E04
:103640001BEC08F02BEC08F0010E0101576F586BD2
:10365000000172EC07F051C056F1110E0101576FD5
:10366000000166EC08F02BEC08F0020E0101576F28
:10367000586B000172EC07F02BEC08F03E520DE1A4
:10368000420E0101616F626B00012DEC05F002C07A
:1036900052F001C051F0010E3E6E030E0101556F54
:1036A000110E546F010E566F0001CCEC08F001C0F2
:1036B00050F0900EF66E080EF76E1BEC08F05052AC
:1036C00009E0020E3E6E036A5050E8BE0306512622
:1036D0000350522252BE05D0525206E1515000080A
:1036E00003E3526A010E516E52BE08D0525203E1FA
:1036F0005150630803E2526A630E516E1CB202D04D
:1037000051C046F01C92DB515E0803E1DC511B08FE
:103710000EE03E5002080AE1420E0101556F576B60
:1037200051C056F1586B000195EC0AF03E6A51EF1A
:1037300021F00101576B586B000172EC07F09A0EF3
:10374000F66E080EF76E1BEC08F0010E0101576FC4
:10375000586B000172EC07F0AC0EF66E080EF76EB7
:10376000060E0101566F0001A5EC07F0020EE96E8E
:1037700052C057F151C056F1B9EC07F02BEC08F0EC
:10378000020E0101576F586B000172EC07F02BEC31
:1037900008F03E520EE1370E0101616F010E626FBB
:1037A00000012DEC05F002C052F001C051F0010EF5
:1037B0003E6E030E0101556F110E546F010E566FD0
:1037C0000001CCEC08F001C050F0B80EF66E080E07
:1037D000F76E1BEC08F0505209E0020E3E6E036AD1
:1037E0005050E8BE030651260350522252AE02D07A
:1037F000526A516A52BE0BD0F851525C08E303E1A1
:103800005150F75D04E2F8C052F0F7C051F052C0D9
:1038100004F151C003F101015AC055F159C054F1EE
:1038200003C100F004C101F05B6B5A6B01C059F198
:1038300000C058F16D6B6C6B5AC06BF159C06AF1E6
:10384000716B706B01C06FF100C06EF100017FEC15
:1038500005F003C057F102C056F101C055F100C098
:1038600054F1D89203C06FF102C06EF101C06DF146
:1038700000C06CF10101736B726B030E716FE80E87
:10388000706F0001ACEC05F001C0EEF000C0EDF08F
:103890001CA613D0EEC002F0EDC001F002320132DE
:1038A00002320132023201C067FF02320230300BB5
:1038B000006E6650CF0B0010666EDB515F0803E1AF
:1038C000DC511B0812E03E5002080CE1370E0101EA
:1038D000556F52C057F151C056F1010E586F00019B
:1038E00095EC0AF03E6A526A516A51EF21F00101EB
:1038F000576B586B000172EC07F0C20EF66E080EA3
:10390000F76E1BEC08F02BEC08F0010E0101576F6D
:10391000586B000172EC07F0D00EF66E080EF76ED1
:10392000060E0101566F0001A5EC07F0020EE96ECC
:1039300052C057F151C056F1B9EC07F02BEC08F02A
:10394000020E0101576F586B000172EC07F02BEC6F
:1039500008F03E520EE13B0E0101616F010E626FF5
:1039600000012DEC05F002C052F001C051F0010E33
:103970003E6E030E0101556F110E546F010E566F0E
:103980000001CCEC08F001C050F0DC0EF66E080E21
:10399000F76E1BEC08F0505209E0020E3E6E036A0F
:1039A0005050E8BE030651260350522252AE02D0B8
:1039B000526A516A52BE0CD05250020809E2FF0A04
:1039C00003E15150E70804E2030E526EE70E516E18
:1039D00052C006F151C005F101015AC055F159C05C
:1039E00054F105C100F006C101F05B6B5A6B01C0D8
:1039F00059F100C058F16D6B6C6B5AC06BF159C036
:103A00006AF1716B706B01C06FF100C06EF1000163
:103A10007FEC05F003C057F102C056F101C055F12B
:103A200000C054F1D89203C06FF102C06EF101C022
:103A30006DF100C06CF10101736B726B030E716F5D
:103A4000E80E706F0001ACEC05F001C0F0F000C0B2
:103A5000EFF01CA413D0F0C002F0EFC001F002326E
:103A6000013202320132023201C067FF02320230FB
:103A7000300B006E6650CF0B0010666EDB51600895
:103A800003E1DC511B0812E03E5002080CE13B0E42
:103A90000101556F52C057F151C056F1010E586FD8
:103AA000000195EC0AF03E6A526A516A51EF21F02A
:103AB0000101576B586B000172EC07F0E60EF66ED1
:103AC000080EF76E1BEC08F02BEC08F0010E01015C
:103AD000576F586B000172EC07F0F40EF66E080E8B
:103AE000F76E060E0101566F0001A5EC07F0010EFE
:103AF000E96E52C057F151C056F1B9EC07F02BEC0A
:103B000008F0020E0101576F586B000172EC07F0CC
:103B10002BEC08F03E520EE13D0E0101616F010EEB
:103B2000626F00012DEC05F002C052F001C051F0AF
:103B3000010E3E6E030E0101556F110E546F010E02
:103B4000566F0001CCEC08F001C050F0000EF66E8C
:103B5000090EF76E1BEC08F0505209E0020E3E6EA3
:103B6000036A5050E8BE030651260350522252AE5B
:103B700002D0526A516A52BE0CD05250020809E279
:103B8000FF0A03E15150E70804E2030E526EE70E0C
:103B9000516E52C008F151C007F101015AC055F1F0
:103BA00059C054F107C100F008C101F05B6B5A6BBA
:103BB00001C059F100C058F16D6B6C6B5AC06BF1CC
:103BC00059C06AF1716B706B01C06FF100C06EF18A
:103BD00000017FEC05F003C057F102C056F101C0AF
:103BE00055F100C054F1D89203C06FF102C06EF1DC
:103BF00001C06DF100C06CF10101736B726B030EBB
:103C0000716FE80E706F0001ACEC05F001C0F2F0CE
:103C100000C0F1F01CA413D0F2C002F0F1C001F01A
:103C20000232013202320132023201C067FF023237
:103C30000230300B006E6650CF0B0010666EDB5109
:103C4000610803E1DC511B0812E03E5002080CE160
:103C50003D0E0101556F52C057F151C056F1010E92
:103C6000586F000195EC0AF03E6A526A516A19D306
:103C70000101576B586B000172EC07F00A0EF66EEB
:103C8000090EF76E1BEC08F02BEC08F0010E010199
:103C9000576F586B000172EC07F051C056F1130ECC
:103CA0000101576F000166EC08F01B0EF66E090E5D
:103CB000F76E070E0101566F0001A5EC07F02BEC23
:103CC00008F0020E0101576F586B000172EC07F00B
:103CD0002BEC08F03E520DE11E0E0101616F626B8C
:103CE00000012DEC05F002C052F001C051F0010EB0
:103CF0003E6E030E0101556F110E546F010E566F8B
:103D00000001CCEC08F001C050F0240EF66E090E54
:103D1000F76E1BEC08F0505209E0020E3E6E036A8B
:103D20005050E8BE030651260350522252AE02D034
:103D3000526A516A52BE05D05250000802E2526ADD
:103D4000516851C04DF0DB51620803E1DC511B08A2
:103D50000EE03E5002080AE11E0E0101556F576B3E
:103D600051C056F1586B000195EC0AF03E6A99D2A9
:103D70000101576B586B000172EC07F02BEC08F057
:103D8000010E0101576F586B000172EC07F02E0E07
:103D9000F66E090EF76E1BEC08F02BEC08F0020E25
:103DA0000101576F586B000172EC07F02BEC08F023
:103DB000030E0101556F546B566B0001CCEC08F0FB
:103DC0002BEC08F06ED20101576B586B000172ECBE
:103DD00007F03C0EF66E090EF76E0A0E0101566FE3
:103DE0000001A5EC07F051C056F1130E0101576F09
:103DF000000166EC08F05D0E01015F6F00017CECD4
:103E000007F02BEC08F0010E0101576F586B000111
:103E100072EC07F02BEC08F0020E0101576F586BA3
:103E2000000172EC07F02BEC08F0030E0101556F56
:103E3000110E546F010E566F0001CCEC08F001C05A
:103E400050F04C0EF66E090EF76E1BEC08F0505257
:103E500007E0036A5050E8BE030651260350522281
:103E600052AE02D0526A516A52BE05D0525000087A
:103E700002E2526A5168DB51640803E1DC511B081D
:103E800003E03E6A51C01EF00CD23E522CE1010EFE
:103E90003E6E1E500F0815E01E50430812E01E50E3
:103EA00051080FE01E5053080CE01E50550809E061
:103EB0001E50570806E01E50600803E01E507F08A1
:103EC00002E21A8C01D01A9C000E1ABC010E0101EC
:103ED000546F1EC061F1626F00012DEC05F002C04D
:103EE00052F001C051F00101576B586B000172ECA8
:103EF00007F0560EF66E090EF76E030E0101566FAF
:103F00000001A5EC07F01EC056F1130E0101576F1A
:103F1000000166EC08F02BEC08F0010E0101576F70
:103F2000586B000172EC07F02BEC08F0020E010157
:103F3000576F040E586F000172EC07F05E0EF66EBC
:103F4000090EF76E060E0101566F0001A5EC07F091
:103F5000000EE96E52C057F151C056F1B9EC07F0AE
:103F60005D0E01015F6F00017CEC07F0030E0101A3
:103F7000556F110E546F010E566F0001CCEC08F016
:103F800001C050F06A0EF66E090EF76E1BEC08F0D9
:103F9000505209E0020E3E6E036A5050E8BE03061E
:103FA00051260350522252AE02D0526A516A52BE7A
:103FB00007D05250000804E21ABC02D0526A51687D
:103FC0001E50430804E152C00AF151C009F1DB510F
:103FD000650803E1DC511B0818E03E5002080FE1C0
:103FE000000E1ABC010E0101546F1EC055F152C0E3
:103FF00057F151C056F1586F000195EC0AF0036A71
:104000001EC051F003C052F03E6A4BD10101576B04
:10401000586B000172EC07F0740EF66E090EF76E25
:104020001BEC08F02BEC08F0030E0101556F110E8C
:10403000546F566B0001CCEC08F001C050F0840EB8
:10404000F66E090EF76E1BEC08F03E5205E1010E0C
:104050003E6E526A516A506E5052D8B485D0036A8F
:104060005050E8BE030651260350522252AE02D0F1
:10407000526A516A52BE08D0525203E15150255C37
:1040800003E225C051F0526A51C01EF0D8901E3490
:104090002A6E010E0101576F586B000172EC07F098
:1040A0007E0E2A240101546F616F010E626F0001C0
:1040B0002DEC05F002C055F101C054F18E0EF66EE4
:1040C000090EF76E040E0101566F0001A5EC07F012
:1040D0001EC056F1110E0101576F000166EC08F089
:1040E000220E01015F6F00017CEC07F0000EE96E0B
:1040F00055C157F154C156F1B9EC07F09A0EF66E5E
:10410000090EF76E040E0101566F0001A5EC07F0D1
:10411000020E0101576F586B000172EC07F0010E9F
:104120001E5C006ED89000360050036A710FE96E75
:10413000000E0320EA6EECCF55F1ED52EFCF54F1B3
:10414000A00EF66E090EF76E040E0101566F000107
:10415000A5EC07F0000EE96E55C157F154C156F1B8
:10416000B9EC07F02BEC08F0DB51660803E1DC51F9
:104170001B081BE03E6A7F0E0101616F626B00014C
:104180002DEC05F002C055F101C054F101010150C0
:10419000700809E1555307E11B0E0001DC6F670E43
:1041A000DB6F03D00101FF0000017BD00101576BE1
:1041B000586B000172EC07F0AA0EF66E090EF76E4E
:1041C0001BEC08F02BEC08F0010E0101576F586B47
:1041D000000172EC07F0B60EF66E090EF76E1BECDE
:1041E00008F02BEC08F03E520DE1010E3E6E5652E7
:1041F00009E15550030806E381BC04D01BB202D08C
:10420000020E3E6E020E0101576F586B000172ECF8
:1042100007F03E50020807E1C40EF66E090EF76E75
:104220001BEC08F006D0D00EF66E090EF76E1BECF4
:1042300008F02BEC08F00101556B110E546F566B12
:104240000001CCEC08F001C050F0DE0EF66E090E55
:10425000F76E1BEC08F050BE18D05050000815E265
:104260003E50020812E1626A040E1F6E010E2A6EB1
:10427000706B6F6B5DEC05F0686B676BDC6B010E50
:10428000DB6F5DEC05F01B8E09D050AE07D03E6AA7
:104290001B0EDC6F580EDB6F526A516A02D0DC6B6A
:1042A000DB6B1F500AE0040AD8B40FEF26F0010AB6
:1042B000D8B45EEF27F061EF27F01AAAD1D01A9A8E
:1042C000030E0101546F56C056F155C055F10A0E48
:1042D000576F0001D5EC06F002C056F001C055F052
:1042E000070E0101546F58C056F157C055F1576B76
:1042F0000001D5EC06F002C058F001C057F058504C
:10430000020807E2FF0A03E15750200802E21D807D
:1043100008D05850010805E303E15750F30801E3C2
:104320001D900B0E0101546F5AC056F159C055F142
:10433000576B0001D5EC06F002C05AF001C059F0ED
:10434000D8905A300101556F5930546F0951542596
:104350000001F76F01010A5155210001F86F0F0E9E
:104360000101546F5CC056F15BC055F1140E576FDC
:104370000001D5EC06F002C05CF001C05BF05550C6
:10438000E1275650E223372A4950375C12E3376A57
:10439000E2C05DF1E1C05CF101015F6B49C05EF11B
:1043A0000001B2EC06F002C0E4F001C0E3F0E26B01
:1043B000E16B1BAA04D01C8E320E4E6E47D01CAE91
:1043C00045D081AA2BD04E5229E04E06456AEF51C6
:1043D000F15D0101546F0001F051F2590101556F77
:1043E000D8905531036E54310001EF250101546F0F
:1043F00003500001F0210101556F553354335533FB
:104400005433553354C167FF55335531300B006E6B
:104410006650CF0B0010666E1AD000011C9EF8C0CB
:1044200002F0F7C001F002320132023201320232F0
:1044300001C067FF02320230300B006E6650CF0BB6
:104440000010666EF8C0FAF0F7C0F9F001014550AF
:10445000030805E181AC03D081AA01D0456A0001BF
:104460001AA60DEF26F01A9681A802D04F5202E04C
:104470001C8C01D01C9C4F5201E04F0601015AC018
:1044800055F159C054F101C100F002C101F05B6B5C
:104490005A6B01C059F100C058F16D6B6C6B5AC07A
:1044A0006BF159C06AF1716B706B01C06FF100C0A4
:1044B0006EF100017FEC05F003C057F102C056F128
:1044C00001C055F100C054F1D89203C06FF102C091
:1044D0006EF101C06DF100C06CF10101736B726B84
:1044E000030E716FE80E706F0001ACEC05F001C0B7
:1044F00000F100C0FFF000C15DF1FFC05CF10101FF
:104500005F6B0A0E5E6F0001B2EC06F001C04AF06C
:104510004A500A0DF350FF5D4B6E1CBE13D0F8C01D
:1045200002F0F7C001F002320132023201320232EF
:1045300001C067FF02320230300B006E6650CF0BB5
:104540000010666E4C2A4C50080801E24C6A1BB6FB
:1045500003D02B5201E02B062D50F55D02E1F653FE
:1045600005E0F66B2DC0F5F0B40E2B6E6251E05DE8
:104570000BE303E16151DF5D07E36151DF5D636FD1
:104580006251E059646F02D0646B636B1BA8BBD0AF
:104590001BAC04D064C066F063C065F081B0B1D0DC
:1045A000E0C05DF1DFC05CF101015F6B640E5E6F26
:1045B0000001B2EC06F002C055F101C054F102C096
:1045C0005BF101C05AF1FEC05DF1FDC05CF1A1ECF0
:1045D00006F002C055F101C054F102C05DF101C006
:1045E0005CF101015F6B0A0E5E6F0001B2EC06F038
:1045F00002C0E8F001C0E7F01BBC39D01B8CE0C062
:104600005DF1DFC05CF101015F6B640E5E6F000164
:10461000B2EC06F002C055F101C054F102C05BF1EA
:1046200001C05AF1FEC05DF1FDC05CF1A1EC06F0E5
:1046300002C055F101C054F102C05DF101C05CF14E
:1046400001015F6B0A0E5E6F0001B2EC06F002C062
:10465000E6F001C0E5F0E0C0D6F0DFC0D5F0E0C084
:1046600062F0DFC061F0E8C0EAF0E7C0E9F0EA51CB
:10467000E85D0DE303E1E751E95D09E2E8C0EAF036
:10468000E7C0E9F0E0C0D6F0DFC0D5F01CD01CBA1E
:1046900015D0640EDF250101546F000E0001E021EA
:1046A0000101556F0001D65D0EE308E1D55101010E
:1046B000545DD8A002D0000106D000011C9AE8C0C9
:1046C000EAF0E7C0E9F0EA51E65D04E30BE1E95105
:1046D000E55D08E25C50020808E2FF0A03E15B5076
:1046E0001F0803E2829881960BD082888186E52B91
:1046F000D8B4E62BE551E95DFB6FE651EA59FC6F52
:1047000002D0829881961BAA2CD11CB2E9D001015B
:104710005AC055F159C054F107C100F008C101F069
:104720005B6B5A6B01C059F100C058F16D6B6C6B3B
:104730005AC06BF159C06AF1716B706B01C06FF1B7
:1047400000C06EF100017FEC05F003C057F102C01C
:1047500056F101C055F100C054F1D89203C06FF179
:1047600002C06EF101C06DF100C06CF10101736B0C
:10477000726B030E716FE80E706F0001ACEC05F008
:1047800001C0F2F000C0F1F001015AC055F159C06A
:1047900054F105C100F006C101F05B6B5A6B01C01A
:1047A00059F100C058F16D6B6C6B5AC06BF159C078
:1047B0006AF1716B706B01C06FF100C06EF10001A6
:1047C0007FEC05F003C057F102C056F101C055F16E
:1047D00000C054F1D89203C06FF102C06EF101C065
:1047E0006DF100C06CF10101736B726B030E716FA0
:1047F000E80E706F0001ACEC05F001C0F0F000C0F5
:10480000EFF0EF51F15D0101546F0001F051F259E9
:104810000101556F576B010E4424016E000E5721A4
:10482000036E01C056F1576F55C15BF154C15AF187
:104830005D6F01C05CF10001A1EC06F002C055F112
:1048400001C054F102C05DF101C05CF101015F6B78
:104850000A0E5E6F0001B2EC06F00150EF25EB6F1F
:104860000250F021EC6F01015AC055F159C054F1CA
:1048700003C100F004C101F05B6B5A6B01C059F138
:1048800000C058F16D6B6C6B5AC06BF159C06AF186
:10489000716B706B01C06FF100C06EF100017FECB5
:1048A00005F003C057F102C056F101C055F100C038
:1048B00054F1D89203C06FF102C06EF101C06DF1E6
:1048C00000C06CF10101736B726B030E716FE80E27
:1048D000706F0001ACEC05F001C0EEF000C0EDF02F
:1048E0001CAC19D040520FE082B00DD082B60BD074
:1048F0005C50010808E303E15B50F30804E38280A5
:10490000828840C043F0DB51D20805E1DC51070842
:1049100002E182861B9C82B602D0829082981CA6FD
:1049200006D04750070803E11C96010E456E1CA4F3
:1049300006D047501E0803E11C94020E456E472A1C
:10494000DB51D1080DE1DC5107080AE14806485265
:1049500007E1DB51D8B4DC07DB071B96526A516ACA
:1049600003D0476A1C941C96425207E042506208EA
:1049700001E342061B84828A09D01B941DA201D048
:10498000829A80B803D01CB001D0829A81B20ED036
:1049900042520CE1DB51D10803E1DC51070808E089
:1049A000DB51D20803E1DC51070802E01CA003D070
:1049B00041C042F01C90435202E0430604D0829072
:1049C0001BB801D082981BBA06D01BB804D08290C5
:1049D0008298819682961CBC07D0DB51D10803E1F6
:1049E000DC51070801E08296DB51D00803E1DC517D
:1049F00007080EE0DB51D10803E1DC51070808E0AD
:104A0000DB51D20803E1DC51070802E08098829470
:104A10006E310101556F00016D310101546F553345
:104A200054333F0E551755C15BF154C15AF15D6BBC
:104A30002CC05CF10001A1EC06F002C055F101C0F0
:104A400054F102C05DF101C05CF101015F6B640EC5
:104A50005E6F0001B2EC06F002C055F101C054F1E6
:104A600002C05BF101C05AF101015D6B0A0E5C6F7F
:104A70000001A1EC06F002C070F001C06FF06E6B97
:104A80006D6BE4510308D8A095D004E1E351FE0812
:104A9000D8A090D0E45304E1E3510F08D8B08AD0F5
:104AA000E431036EE331026E03320232033202322A
:104AB000033202320F0E031602C024F02550245C8C
:104AC00074E2010E245C006ED89000360050036A38
:104AD000710FE96E000E0320EA6EECCF55F1ED5236
:104AE000EFCF54F1D8902434036A710FE96E000EB1
:104AF0000320EA6EECCF57F1ED52EFCF56F1010EE5
:104B0000245C006ED89000360050036A710FE96E85
:104B1000000E0320EA6EECCF03F0ED52EF500101DE
:104B2000565F0350575B57C15BF156C15AF15D6B3D
:104B30000A0E5C6F0001A1EC06F002C057F101C043
:104B400056F10101573356335733563357335633E3
:104B5000573356330F0E57170001E3510F0B006EFA
:104B6000E8CF58F10101596B57C15BF156C15AF1B9
:104B70005D6B5C6F0001A1EC06F002C057F101C053
:104B800056F102C05DF101C05CF101015F6B0A0EDC
:104B90005E6F0001B2EC06F00150010154255F6E1A
:104BA000025055210001606F04D06AC060F069C0F6
:104BB0005FF002D0606B5F6A60C05DF15FC05CF166
:104BC00001015F6B640E5E6F0001B2EC06F002C083
:104BD00055F101C054F102C05BF101C05AF101016D
:104BE0005D6B640E5C6F0001A1EC06F002C0E0F0AA
:104BF00001C0DFF0DF515F5C0101546F0001E05143
:104C000060590101556F555303E15451320806E2D2
:104C1000320E0001DF27000EE023010154D11AAA51
:104C20002BD01A9A030E0101546F56C056F155C08D
:104C300055F10A0E576F0001D5EC06F002C056F090
:104C400001C055F05550E1275650E223372A37501E
:104C5000040812E2376AE2C05DF1E1C05CF10101D3
:104C60005F6B050E5E6F0001B2EC06F002C0E4F06F
:104C700001C0E3F0E26BE16B1AA61ED11A96672B16
:104C8000D8B4682BE451030802E2E46BE36B010142
:104C9000576B586B000172EC07F0F00EF66E090EC0
:104CA000F76E030E0101566F0001A5EC07F0020E2E
:104CB000E96EE4C057F1E3C056F1B9EC07F0F70E26
:104CC000F66E090EF76E050E0101566F0001A5EC98
:104CD00007F0000EE96E68C057F167C056F1B9ECF5
:104CE00007F081BCB3D01BAEB1D0E431036EE33129
:104CF000026E0332023203320232033202320F0EEC
:104D0000031602C024F02A50245CD8A09ED02A2A80
:104D100068C06CF067C06BF0010E0101576F586BF3
:104D2000000172EC07F0800E6F250101546F000E38
:104D3000000170210101556F020EF66E0A0EF76E2A
:104D4000050E566F0001A5EC07F0010EE96E55C186
:104D500057F154C156F1B9EC07F0200E01015F6F15
:104D600000017CEC07F02BEC08F0800E6F250101B0
:104D7000546F000E000170210101556F67C056F19C
:104D8000F250006EF29E54C1A9FF56C1A8FFA69C26
:104D9000A69EA6840F01550EA76EAA0EA76EA68228
:104DA000A6B2FED7A6940050F212810E00016F2524
:104DB0000101546F000E000170210101556F68C0A0
:104DC00056F1F250006EF29E54C1A9FF56C1A8FFE1
:104DD000A69CA69EA6840F01550EA76EAA0EA76ECE
:104DE000A682A6B2FED7A6940050F212020E0001CF
:104DF0006F27000E7023020E0101576F586B0001E0
:104E000072EC07F0010E2A5C0101546F566F130E0D
:104E1000576F000166EC08F0110EF66E0A0EF76E81
:104E20000C0E0101566F0001A5EC07F02BEC08F009
:104E3000030E0101576F586B000172EC07F01E0E54
:104E4000F66E0A0EF76E1BEC08F036D01BAE34D0AF
:104E50000F0E0101556F6CC057F16BC056F1010E7A
:104E6000586F000195EC0AF0010E2A5C0101546FA5
:104E70000E0E556F576B54C156F1586B000195ECEF
:104E80000AF07F0E0101556F576B566B586B00018E
:104E900095EC0AF00E0E0101616F626B00012DECC2
:104EA00005F001C025F05DEC05F01F6A1B0EDC6FFC
:104EB0005C0EDB6F3E6A1B9E010105D0010103D031
:0E4EC00000011F6A01010001D3EF0DF0030095
:0200000400F00A
:1000000000000000000000000000000000000000F0
:1000100000000000000000000000000000000000E0
:1000200000000000000000000000000000000000D0
:1000300000000000000000000000000000000000C0
:1000400000000000000000000000000000000000B0
:1000500000000000000000000000000000000000A0
:100060000000000000000000000000000000000090
:100070000000000000000000000000000000000080
:100080000000000000000000000000000000000070
:100090000000000000000000000000000000000060
:1000A0000000000000000000000000000000000050
:1000B0000000000000000000000000000000000040
:1000C0000000000000000000000000000000000030
:1000D0000000000000000000000000000000000020
:1000E0000000000000000000000000000000000010
:1000F0000000000000000000000000000000000000
:020000040030CA
:0E00000000E31E3F00BF810000800FE00F40B4
:00000001FF
